:020000040000FA
:020000003628A0
:08000800CE00030ECF008312AD
:100010008B1C0B288B1081010B114F0E8300CE0E11
:100020004E0E09000F398207AF29B829BE29C4290D
:10003000CA29D029D629DC29E229E829EE29F42980
:10004000FA29AF29AF29AF290F398207072B082BCF
:100050000F2B162B1D2B1E2B232B2A2B2B2B312B3F
:10006000382B422B422B422B422B422B8316FF2351
:10007000900083163F3085003F3087008312FF30A9
:100080008500FF3087008312073099008316003007
:1000900091008316C83081008312013090008316CE
:1000A00000308C00831210308B00203084008001DF
:1000B000840A60300402031C572881018E018F01DD
:1000C0000B118B100B108C01FF30C4008030BF006F
:1000D000C0010430C300A20158226400C408031DFB
:1000E00077288030BF00C0010430C300C40AC30BAE
:1000F00094280430C300440FC40A44082F3C031C56
:10010000922803103F0CCC00400CCD000310CC0C07
:10011000CD0C0310CC0C4D0CC0024C08031C013E4E
:10012000BF029428BF01C0014008003CC2003F0844
:10013000031C3F0A803CC10000000F080F3C03185D
:100140009D288F0158222F08BC003508BD002908C2
:10015000BB00F2203B08A9003D08B5003C08AF00F9
:100160003008BC003608BD002A08BB00F2203B085E
:10017000AA003D08B6003C08B0003108BC003708B2
:10018000BD002B08BB00F2203B08AB003D08B700C8
:100190003C08B1003208BC003808BD002C08BB0088
:1001A000F2203B08AC003D08B8003C08B200330820
:1001B000BC003908BD002D08BB00F2203B08AD0093
:1001C0003D08B9003C08B3003408BC002E08BB0051
:1001D0003E213B08AE003C08B40044084B3C031CE5
:1001E0007E226E283B0800380319080012203D1DAE
:1001F00003293F08CA004008CB004A04031D142904
:10020000BB01BD010800BD1C08293E08C900262904
:100210003D1C13294108CA004208CB003F08400496
:100220000319BD14142908003E0807224030CA07EC
:10023000003003180130C9070318C9034A08BC0776
:10024000003003180130C9070318C903C90803198E
:100250000800831628088500C90B2C29FF3085006B
:100260008312FF3085008316D8308500FF3085006B
:100270008312080012203E08C900262900380319FD
:1002800008001220C608031D4B293E08C700C801FC
:100290000430C500C60AC50B68290430C500460FE6
:1002A000C60A46082F3C031C66290310470CCC00E5
:1002B000480CCD000310CC0CCD0C0310CC0C4D0C15
:1002C000C8024C08031C013EC7026829C701C801C7
:1002D0003A1973294808003CCA004708031C470A1A
:1002E0003E02C90077294808CA004708C9004908E2
:1002F000031D7E294A08403C031893294A08BC077D
:10030000003003180130C9070318C9033A0805393A
:10031000013A031D92293A154A08C8004908C70046
:100320000130C60026214608483C031808003A0858
:100330000539053A031DA029BB01BA01C601080011
:100340003A080639023A031908000430BA06C60111
:1003500008001220831628088500831208008316DF
:10036000FF3085008312FF3085000030BE0008009A
:10037000FC30A800FD3085000130002AFC30A800C8
:10038000FE3085000230002ADD30A800DF30850015
:100390000330002ADD30A800FD3085000430002A3B
:1003A000DB30A800FB3085000530002ADB30A800D8
:1003B000DF3085000630002AFA30A800FE308500C4
:1003C0000730002AFA30A800FB3085000830002AE8
:1003D000DE30A800DF3085000930002ADE30A800BA
:1003E000FE3085000A30002AF930A800FD30850073
:1003F0000B30002AF930A800FB3085000C30002AB1
:1004000083169B001C141A088312BE000800C90141
:10041000CA0CCB0C0318C907C90CCA0CCB0C0318A7
:10042000C907C90CCA0CCB0C0318C907C90CCA0CE4
:10043000CB0C0318C907C90CCA0CCB0C0318C9078D
:10044000C90CCA0CCB0C0318C907C90CCA0CCB0CBD
:100450000318C907C90CCA0CCB0C0318C907C90C6F
:10046000CA0CCB0C0318C907C90CCA0CCB0C031857
:10047000C907C90CCA0CCB0C0318C907C90CCA0C94
:10048000CB0C0318C907C90CCA0CCB0C0318C9073D
:10049000C90CCA0CCB0C0318C907C90CCA0CCB0C6D
:1004A0000318C907C90CCA0CCB0C0318C9070800EC
:1004B00007083F3A3F39A300851D2317051EA317E0
:1004C0008722A3002308031D692AA6030319A40198
:1004D000080023082502031D6F2AA4010800230831
:1004E00024020319772A0330A7002308A4000A3046
:1004F000A600A70B08002408A5000800250803197A
:100500000800220203190800C4012508C02A230894
:100510000319003496220038031DA000B0220038D1
:10052000031DA1002008201E210708002308083A07
:10053000F839031910342308403AF0390319043408
:100540002308603AB039031908342308183A90395F
:10055000031918342308883A8039031914340034F5
:100560002308043A0739031901342308023A0339EE
:10057000031903342308013A013903190234003402
:1005800022081C39031DD42AB701B801B901031090
:10059000250CCA0003104A0C043E24200330A20597
:1005A00025081C39A204F22A220825061C39031941
:1005B000F22A22082504CA004A1EC52A2208250557
:1005C000CA004A1EED2A22080C390319C52A2B231A
:1005D000220803391038A200F22A371538153915C8
:1005E0000330A20522080339031DFD2A250803391B
:1005F000242025080339A204062B220825060339E6
:100600000319062B351536151C30A2050800080005
:100610000830A9000C30AA00351436140800073041
:10062000A9000B30AA003514361408000730A900C1
:100630000C30AA0035143614080008000A30AB004C
:100640003714381508000A30AB000230AC003714FC
:100650003814080008000930AB0037143815391574
:1006600008000930AB000130AC0037143814080022
:100670000930AB000430AC000330AD00371438143F
:0606800039140800080017
:084000000F000F000F000F007C
:02400E00C43FAD
:1042000000004000400040004000400040003000FE
:0A4210004000400030003000400084
:00000001FF
